:020000040000FA
:02000000092ACB
:08000800A000030E8312A10009
:100010002608820020342034203420342034203438
:100020006534733463342E34613473346D34203466
:10003000563431342E3435342034203420342034B6
:100040004534533443344334203420342034203472
:10005000B801B901BA01B90AB601B7010310B50D6B
:10006000B80D03183628B90DBA0D2E28B80CB50CEA
:100070003508B3023808031C013EB402031C4C28A7
:100080003908B6043A08B7040310BA0CB90C0318BF
:100090000800B80CB50C38283508B3070318B40AA3
:1000A0003808B4074428B601B7013508B800381C31
:1000B0005F283308B60734080318013EB70703105A
:1000C000B80C3808031908000310B30DB40D5728F5
:0C00D000313E8200713E8200B13E820091
:1002000085010000062A27088500082200008501D4
:10021000062A2708850005292708850000000B29E4
:10022000270885000E2927088500000012292708C5
:100230008500152927088500000019292708850051
:1002400000001C2927088500042A000085010822D7
:10025000292927088500042A000085010822302961
:100260002729003400340034033409340C341034AA
:10027000133417341A341E34F134F134F134F134B8
:10028000F134F134F134F134F134F134F134F13446
:10029000F134F134F134F134F134F134F134F13436
:1002A000F134F134F134F134F134F134F134F13426
:1002B000F134F134F134F134F134F134F134F13416
:1002C000F134F134F134F134F134F134F134F13406
:1002D000F134F134F134F134F134F1342C34253487
:1002E000223400340034003400340034003400344C
:1002F0000034003400340034FB34FA34F834F7347A
:10030000F534F334F134EF34ED34EB34E934E734DD
:10031000E434E234DF34DC34D934D634D234CF346C
:10032000CB34C734C334BE34B934B434AE34A83457
:10033000A1349A34923489347F34753469345C340E
:100340004D343C3429341334093409340934093424
:1003500009340934093409340934093408340834B7
:100360000834083408340834C834C834C834C834AD
:10037000C834C834C834C834C934C934C934C93499
:10038000C934C934C934C934C934C934C934C93485
:10039000C934C934C934C934C934C934C934C93475
:1003A000C934C934C934C934C934C934C934C93465
:1003B000C934C934C934C934C934C934C934C93455
:1003C000C934C934C934C934CD34D334D934DE3412
:1003D000E434E934EE34F334F834FC3400340034DB
:1003E0000034A218F829A214000085012908FD296B
:1003F000270885002808A210000081000B11210E9B
:100400008300A00E200E09002808FD292908FD29D7
:1004100008008316FF239000831201308A008501B3
:100420008316303001389F00103095000030810075
:10043000DF30FB3985008312FF3081008B160130DD
:100440009F00A2011430A300A501A701A801A901E2
:10045000F130A600FF30AF00B000B100B2008B1742
:10046000EA222218302A4308BC00BE004208BB0022
:10047000403EBD000318BE0AEA2222183C2A420868
:100480003D024308031C013E3E0203183C2A420879
:10049000BD004308BE003B083D02B300AD003C0870
:1004A000031C013E3E02B400AE004030B5002820DF
:1004B0003608AC00B300B40153203608AD0237084B
:1004C000031C013EAE020310AE0CAD0C3B08AD07A1
:1004D0003C080318013EAE07EA2222186C2A3D08A8
:1004E00042023E08031C013E43020318472A420809
:1004F000B3004308B40015230038031D6C2A8B1782
:10050000D022DD22D0228B17A501A701C02223080B
:10051000A4000E232218872A6820003C031D872A86
:10052000A40B892A0130A300A7018501A501C022DF
:100530002030A7000E232218842A25020319AC2A92
:100540000318A62AA50AC02222119A2A221DAA2A25
:10055000A502C02222159A2A22112608003C031D5A
:100560009A2A851D9A2A0430A7003F30A500C02290
:100570000E232218842A6820003C031D942AB82ADE
:1005800025086A20AA0025086C20AB0025086820F1
:100590008B12A6002A08A8002B08A9008B160800B9
:1005A000C830BF0020308500082208220822082217
:1005B0008501E322BF0BD22A0800C830BF00E32226
:1005C000BF0BDF2A080064003230C0000822C00BD5
:1005D000E62A08002923221808000530C1000E0869
:1005E000C2000F08C3002923221808004208FD3E5C
:1005F000B3004308031CFF3EB40033080E02B300EF
:100600003408031C013E0F02B400031DEA2A073020
:1006100033020318EA2AC10BF32A080029232218FF
:1006200000340E08B3000F08B4002D08B3022E08E2
:10063000031C013EB402031C00342C08B500282022
:10064000B708031D3F344030360203183F343608E4
:10065000080022104030C4001B30C5008E018F01FD
:10066000413090005623221800340E080F0403195D
:10067000322B03309F0056232218003409300F021A
:100680000318502B051E3B2B90019F185B2B5D23FD
:10069000553C03185B2B03300F02031C2E2B080064
:1006A000562322180034051E502B2E2B6400C40B39
:1006B0000800C50B0800221408003108B2003008F9
:1006C000B1002F08B0001E08AF00C600C7013008F7
:1006D000C6070318C70A3108C6070318C70A320835
:1006E000C6070318C70AC70CC60CC70CC60C4608B9
:0206F000080000
:02400E00CC3FA5
:00000001FF
